:100000000C9428120C9468120C9468120C946812C8
:100010000C9468120C9468120C9468120C94681278
:100020000C9468120C9468120C9468120C94681268
:100030000C9468120C9468120C9468120C94681258
:100040000C9468120C94191C0C9468120C9468128D
:100050000C9468120C94241B0C9468120C946897EE
:100060000C9468120C94743B0C943E3B0C946812F4
:100070000C9468120C9468120C9468120C94681218
:100080000C9468120C9468120C9468120C94681208
:100090000C9468120C9468120C9468120C946812F8
:1000A0000C9468120C9468120C9468120C946812E8
:1000B0000C9468120C9468120C9468120C946812D8
:1000C0000C9468120C9468120C9468120C946812C8
:1000D0000C9468120C9468120C9468120C946812B8
:1000E0000C946812084AD73B3BCE016E84BCBFFD1E
:1000F000C12F3D6C74319ABD56833DDA3D00C77FF8
:1001000011BED9E4BB4C3E916BAAAABE0000008090
:100110003F05A84CCDB2D44EB93836A9020C50B91F
:10012000918688083CA6AAAA2ABE000000803F004B
:100130004E414E494E495459494E46CDCCCC3D0ACC
:10014000D7233C17B7D13877CC2B329595E6241FAF
:10015000B14F0A000020410000C84200401C462068
:10016000BCBE4CCA1B0E5AAEC59D7400407A10F33B
:100170005A00A0724E18090010A5D4E80000E876D5
:1001800048170000E40B54020000CA9A3B0000002C
:10019000E1F505000080969800000040420F000045
:1001A00000A08601000000102700000000E8030006
:1001B0000000006400000000000A000000000001D0
:1001C00000000000002C76D888DC674F0823DFC1D0
:1001D000DFAE59E1B1B796E5E3E453C63AE651998B
:1001E0007696E8E6C28426EB898C9B62ED407C6FB4
:1001F000FCEFBC9C9F40F2BAA56FA5F490055A2A6B
:10020000F75C936B6CF9676DC11BFCE0E40D47FE76
:10021000F520E6B500D0ED902E030094357705006B
:1002200080841E080000204E0A000000C80C3333F2
:1002300033330F986E12831141EF8D2114893BE601
:100240005516CFFEE6DB18D1844B381BF77C1D908A
:100250001DA4BBE424203284725E228100C9F124F3
:10026000ECA1E53D27434F4D4D554E49434154497F
:100270004F4E0044525952554E004552524F525320
:1002800000494E464F004543484F004D323400531D
:10029000544F505045442E20005072696E74657260
:1002A0002073746F707065642064756520746F20AE
:1002B0006572726F72732E204669782074686520AB
:1002C0006572726F7220616E6420757365204D399E
:1002D000393920746F20726573746172742E20280E
:1002E00054656D70657261747572652069732072F2
:1002F000657365742E20536574206974206166747B
:1003000065722072657374617274696E67290A0080
:100310004E6F20436865636B73756D2077697468F1
:10032000206C696E65206E756D6265722C204C6163
:100330007374204C696E653A20004E6F20436865E7
:10034000636B73756D2077697468206C696E6520C6
:100350006E756D6265722C204C617374204C696EF1
:10036000653A2000636865636B73756D206D697312
:100370006D617463682C204C617374204C696E65E8
:100380003A20004C696E65204E756D626572206979
:1003900073206E6F74204C617374204C696E6520FD
:1003A0004E756D6265722B312C204C617374204C3C
:1003B000696E653A20004D313130005365726961D4
:1003C0006C20737461747573206D69736D617463EF
:1003D000680A0053442072656164206572726F720E
:1003E0000A00746F6F206D75636820696E616374B5
:1003F0006976652074696D65202D2063757272655C
:100400006E7420636F6D6D616E643A20002121204F
:100410004B494C4C20636175736564206279200000
:100420004D6564696120496E73657274656400622C
:100430007573793A2070617573656420666F7220F8
:10044000696E7075740A00627573793A207061750F
:1004500073656420666F7220757365720A00627539
:1004600073793A2070726F63657373696E670A00FF
:100470006563686F3A004572726F723A002F2F61A0
:100480006374696F6E3A006E6F7469666963617454
:10049000696F6E20006E6F74696669636174696F5D
:1004A0006E2000656E6400627574746F6E00486F34
:1004B00074656E6420746F6F20636F6C640A0070E3
:1004C000617573656400486561642063616E6E6F79
:1004D00074206265207061726B6564005061757391
:1004E000650020440020204D323030205300202869
:1004F00044697361626C6564293A0046696C616D98
:10050000656E742073657474696E67730020204D86
:100510003230312058004D617820416363656C654D
:10052000726174696F6E2028756E6974732F7332EF
:10053000290020204D3230332058004D617820664C
:1005400065656472617465732028756E6974732FB4
:1005500073290020520020204D32303420500041B9
:100560006363656C65726174696F6E2028756E696E
:1005700074732F7332292028503C7072696E742D69
:10058000616363656C3E20523C7265747261637492
:100590002D616363656C3E20543C74726176656CBA
:1005A0002D616363656C3E2900204A0020540020C1
:1005B000530020204D323035204200416476616E78
:1005C0006365642028423C6D696E5F7365676D6585
:1005D0006E745F74696D655F75733E20533C6D6921
:1005E0006E5F66656564726174653E20543C6D693A
:1005F0006E5F74726176656C5F6665656472617466
:10060000653E204A3C6A756E635F6465763E2900EC
:1006100020440020490020204D3330312050004834
:100620006F74656E642050494400204400204900E6
:1006300020204D333034205000426564205049441E
:100640000020440020204D35393320592046002019
:10065000440020204D3539332058204600496E7023
:1006600075742053686170696E6700203B002055E7
:100670000020204D363033204C0046696C616D659A
:100680006E74206C6F61642F756E6C6F61640020F6
:10069000496E76616C696420657874727564657200
:1006A0002000536C6565702E2E2E0070726F6D7079
:1006B000745F00626567696E004D302053746F701F
:1006C000004D312053746F70004E6F204D6F766572
:1006D0002E00456E642066696C65206C6973740A2F
:1006E00000426567696E2066696C65206C69737489
:1006F0000A004E6F206D656469610A0053442063EF
:100700006172642072656C65617365640A0072656C
:1007100073756D6500526573756D696E672053441E
:1007200000286E6F2066696C6529004375727265DA
:100730006E742066696C653A20002E0A0044656C70
:100740006574696F6E206661696C65642C2046690A
:100750006C653A200046696C652064656C6574655B
:10076000643A0043616E6E6F74206F70656E207323
:10077000756264697220002569730025696D202502
:100780006973002569682025696D20256973002536
:100790006964202569682025696D20256973002515
:1007A000697920256964202569682025696D2025DF
:1007B0006973005072696E742074696D653A200027
:1007C0006F6B006F666600860281027A02730265B3
:1007D0000244454255473A004D31313320530047DA
:1007E000656E697573204F46462E007D7D7D0A003B
:1007F0002C7A3A002C793A007D2C6D61783A7B781E
:100800003A002C7A3A002C793A007D7D2C776F7271
:100810006B3A7B6D696E3A7B783A002C7A3A002C01
:10082000793A007D2C6D61783A7B783A002C7A3ADF
:10083000002C793A00617265613A7B66756C6C3A9E
:100840007B6D696E3A7B783A00434F4E4649475F6D
:100850004558504F5254004D4541545041434B0070
:10086000434F4F4C45525F54454D504552415455AE
:100870005245004348414D4245525F54454D504515
:1008800052415455524500424142595354455050EB
:10089000494E470041524353004D4F54494F4E5F1C
:1008A0004D4F44455300544845524D414C5F5052C2
:1008B0004F54454354494F4E00455854454E4445C6
:1008C000445F4D323000435553544F4D5F464952BB
:1008D0004D574152455F55504C4F4144004C464E98
:1008E0005F5752495445004C4F4E475F46494C456F
:1008F0004E414D45004155544F5245504F52545F63
:1009000053445F5354415455530053445F57524925
:10091000544500524550454154004D554C54495F93
:10092000564F4C554D45005344434152440050529C
:100930004F4D50545F535550504F525400484F53F1
:10094000545F414354494F4E5F434F4D4D414E44D8
:100950005300454D455247454E43595F5041525310
:10096000455200434153455F4C494748545F42520A
:10097000494748544E45535300544F47474C455FF1
:100980004C494748545300534F4654574152455FD2
:10099000504F574552004255494C445F50455243D1
:1009A000454E54004C4556454C494E475F444154D2
:1009B00041005A5F50524F42450052554E4F5554D8
:1009C000004155544F4C4556454C005052494E54E9
:1009D0005F4A4F420050524F4752455353004155D2
:1009E000544F5245504F52545F54454D500041555D
:1009F000544F5245504F52545F504F5300564F4C36
:100A0000554D455452494300454550524F4D0042C3
:100A1000494E4152595F46494C455F5452414E53ED
:100A20004645520053455249414C5F584F4E5F581E
:100A30004F4646004649524D574152455F4E414D43
:100A4000453A4D61726C696E20322E312E322E3154
:100A500020284F6374203133203230323320313438
:100A60003A33393A35302920534F555243455F4385
:100A70004F44455F55524C3A6769746875622E63FE
:100A80006F6D2F4D61726C696E4669726D77617220
:100A9000652F4D61726C696E2050524F544F434F19
:100AA0004C5F56455253494F4E3A312E30204D41FE
:100AB0004348494E455F545950453A47656E6975FC
:100AC000732045585452554445525F434F554E5438
:100AD0003A3120555549443A63656465326132665E
:100AE0002D343161322D343734382D396231322D85
:100AF000633535633632663336376666002F2F002E
:100B00003F4A206F7574206F662072616E676520A2
:100B100028302E303120746F20302E33290A0020E7
:100B200058004F4646004F4E003B200020204D61AC
:100B3000783A2000200020204D696E3A2000203BAA
:100B4000200020204D323131205300250A0046522A
:100B50003A0020466C6F773A200064697300656E36
:100B60000043290A0061626C656420286D696E206B
:100B700074656D702000436F6C64206578747275C5
:100B80006465732061726520004F666673657473D7
:100B9000204170706C69656400546F6F20666172EB
:100BA0002066726F6D207265666572656E63652082
:100BB000706F696E740A00454550524F4D204F4B7F
:100BC0000A00206F72203020746F206469736162A4
:100BD0006C650A003F4672657175656E6379202801
:100BE0004629206D75737420626520677265617493
:100BF0006572207468616E20003F5A657461202818
:100C000044292076616C7565206F7574206F6620AD
:100C100072616E67652028302D31290A004D383405
:100C2000005072696E7420446F6E6500446F6E658B
:100C3000207072696E74696E672066696C650A005F
:100C40004D3737004D333100496E76616C69642051
:100C500065787472756465720A0020204D323036F2
:100C6000205800486F6D65206F6666736574004498
:100C70006966663A2020200046726F6D5374703AA0
:100C800000537465707065723A005261773A2020A3
:100C90002020000A4C6F676963616C3A00436F75EE
:100CA0006E7420453A004361703A0047322F473353
:100CB0002062616420706172616D65746572730A8F
:100CC0000020573A0042656420436F6F6C696E677D
:100CD0002E2E2E004265642048656174696E672E71
:100CE0002E2E00206661696C6564212042616420BB
:100CF0006865617465722069640A00504944204146
:100D000075746F74756E650023646566696E652021
:100D100044454641554C545F0000626564004B6495
:100D200020004B6920004B7020005049442074750E
:100D30006E696E6720646F6E65002066696E697308
:100D4000686564212050757420746865206C617337
:100D500074204B702C204B6920616E64204B642002
:100D6000636F6E7374616E74732066726F6D206250
:100D7000656C6F7720696E746F20436F6E6669676C
:100D800075726174696F6E2E680A00504944204183
:100D900075746F74756E6500206661696C65642199
:100DA0002074696D656F75740A005049442041755F
:100DB000746F74756E65004175746F74756E65201F
:100DC0006661696C6564212054696D656F75742E68
:100DD00000206661696C6564212054656D706572E0
:100DE000617475726520746F6F20686967680A00A6
:100DF000504944204175746F74756E6500204B64D2
:100E00003A2000204B693A2000204B703A20002005
:100E1000436C617373696320504944200A00204E7B
:100E20006F206F76657273686F6F740A0020547557
:100E30003A2000204B753A2000206D61783A20005E
:100E4000206D696E3A200020643A200020626961BA
:100E5000733A200048656174696E672E2E2E00205B
:100E600073746172740A00504944204175746F7440
:100E7000756E65004175746F74756E652066616985
:100E80006C6564212054656D70657261747572655E
:100E900020746F6F20686967682E00206661696C36
:100EA0006564212054656D7065726174757265208A
:100EB000746F6F20686967680A0050494420417563
:100EC000746F74756E6500504944204175746F7479
:100ED000756E6500486F6D696E67204661696C6567
:100EE00064006F70656E005452494747455245444F
:100EF000003A20007A5F6D696E00795F6D696E005F
:100F0000785F6D696E005265706F7274696E6720EC
:100F1000656E6473746F70207374617475730A0006
:100F200020746F6F206C6F6E6720657874727573B4
:100F3000696F6E2070726576656E7465640A002054
:100F4000636F6C6420657874727573696F6E20705E
:100F5000726576656E7465640A00000000C000006A
:100F6000A0C0000000005761726E696E673A2048A9
:100F70006F6D696E672042756D7020446976697384
:100F80006F72203C20310A0002020400005E430020
:100F9000006B4300007A430000A0400000A0400026
:100FA000000040000000010000000100008000552A
:100FB0005555000000400033333300AAAA2A0049E7
:100FC00092240000002000C7711C0099991900D1DB
:100FD000451700555515003BB11300244912001167
:100FE000111100000010000F0F0F00E3380E004336
:100FF000790D00CCCC0C00C3300C00E8A20B0064CF
:10100000210B00AAAA0A00703D0A009DD8090042DF
:101010007B090092240900DCD308008888080010AE
:1010200042080000000800F0C1070087870700752C
:10103000500700711C07003EEB0600A1BC060069CA
:1010400090060066660600703E06006118060017EE
:10105000F4050074D105005BB00500B29005006294
:101060007205005555050078390500B81E050005C4
:101070000505004EEC040087D40400A1BD040090D7
:10108000A7040049920400C17D0400EE690400C772
:10109000560400444404005C32040008210400416A
:1010A000100400000004003FF00300F8E0030026F5
:1010B000D20300C3C30300CCB503003AA803000A5F
:1010C0009B0300388E0300C08103009F750300D08E
:1010D000690300505E03001D530300344803009170
:1010E0003D03003333030016290300381F03009724
:1010F000150300300C0300030303000BFA02004940
:10110000F10200BAE802005CE002002DD802002DD6
:10111000D0020059C80200B0C0020031B90200DAA2
:10112000B10200AAAA0200A0A30200BC9C0200FA1D
:101130009502005C8F0200DF880200828202004577
:101140007C02002776020027700200436A02007CBE
:10115000640200D05E02003F590200C8530200FF43
:10116000FDFCFAF8F6F4F2F0EEECEAE9E7E5E3E18B
:10117000E0DEDCDAD9D7D5D4D2D0CFCDCBCAC8C740
:10118000C5C3C2C0BFBDBCBAB9B7B6B4B3B2B0AFC5
:10119000ADACAAA9A8A6A5A4A2A1A09E9D9C9A991F
:1011A000989795949392908F8E8D8B8A8988878655
:1011B00084838281807F7E7D7B7A7978777675746F
:1011C000737271706F6E6D6C6B6A69686766656467
:1011D000636261605F5E5D5C5B5A59585857565553
:1011E0005453525150504F4E4D4C4B4A4A49484728
:1011F0004646454443424241403F3E3E3D3C3B3BE8
:101200003A39383837363535343332323130302F99
:101210002E2E2D2C2B2B2A2929282727262525243D
:10122000232322212120201F1E1E1D1C1C1B1B1AD4
:10123000191918181716161515141313121211115F
:10124000100F0F0E0E0D0D0C0C0B0A0A09090808E1
:101250000707060605050404030302020100000057
:10126000005C430000664300007A43000000C000B9
:1012700000A0C00000000053657474696E6773209D
:1012800053746F72656400290A0020627974657373
:101290003B20637263200053657474696E6773202A
:1012A00053746F726564202800454550524F4D209D
:1012B000496E697469616C697A65640A0048617293
:1012C00064636F6465642044656661756C74205363
:1012D000657474696E6773204C6F61646564002087
:1012E000286D6D290020204D3134392043203B20CA
:1012F000556E69747320696E2043656C73697573EC
:101300000A0054656D706572617475726520556E62
:10131000697473002020473231203B004C696E65B0
:10132000617220556E69747300454550524F4D20CF
:101330006461746173697A65206572726F722E0AD6
:10134000004572723A20454550524F4D204352435A
:1013500000202863616C63756C6174656429210ADF
:101360000020213D2000454550524F4D204352431F
:10137000206D69736D61746368202D202873746F0C
:10138000726564292000454550524F4D20436F72CD
:10139000727570740A002053697A653A2000496EAC
:1013A0006465783A200053746F72656420736574C5
:1013B00074696E677320726574726965766564001E
:1013C000290A002062797465733B206372632000F0
:1013D0002073746F7265642073657474696E6773CB
:1013E0002072657472696576656420280000009635
:1013F000430000964300004842000020420000A045
:10140000420000A0420000C8430080DE43D0070035
:1014100000D00700006400000010270000204D618C
:10142000726C696E3D563838290A00454550524F56
:101430004D2076657273696F6E206D69736D61748E
:1014400063682028454550524F4D3D0020436F753D
:101450006E7420583A00004500626564002C2073C9
:10146000797374656D2073746F70706564212048A2
:1014700065617465725F49443A20004572723A2092
:101480004D415854454D50004D415854454D502004
:101490007472696767657265640048656174696E36
:1014A00067204661696C65640048656174696E67B0
:1014B000206661696C6564004D353234004D313110
:1014C000322053687574646F776E004572723A20EB
:1014D0004D494E54454D50004D494E54454D5020B8
:1014E00074726967676572656400544845524D417E
:1014F0004C2052554E4157415900546865726D61F8
:101500006C2052756E6177617900202F0020424077
:101510003A0020403A0020573A0020583A00205321
:10152000004D3130362050000000210024002700FB
:101530002A002D00300033000101000004010701E2
:101540000A017C3C3E5E2B3D3F2F5B5D3B2C2A22FB
:101550005C0043616E6E6F74206F70656E207375F2
:1015600062646972200053442063617264206F6B6F
:101570000A006F70656E526F6F74206661696C65EA
:10158000640A00766F6C756D652E696E69742066ED
:1015900061696C65640A004E6F2053442063617278
:1015A000640A002E0A006F70656E206661696C65C2
:1015B000642C2046696C653A200046696C6520738E
:1015C000656C65637465640A002053697A653A2026
:1015D0000046696C65206F70656E65643A20004551
:1015E0004E4420535542524F5554494E450A00220D
:1015F00020706F73002220706172656E743A220051
:10160000535542524F5554494E452043414C4C206E
:101610007461726765743A220053756263616C6C21
:10162000204F766572666C6F7700457863656564F8
:101630006564206D617820535542524F5554494E90
:10164000452064657074683A0057726974696E6702
:1016500020746F2066696C653A20004E6F742053C9
:1016600044207072696E74696E670A00534420707A
:1016700072696E74696E67206279746520006672A3
:1016800065736800646F696E67002066696C653A0F
:1016900020004E6F7720000A4D3234004D32332047
:1016A0002573002F6175746F25632E670070012C00
:1016B0000190012701B0012201C0011D01F00118B4
:1016C000011002130130020E0160020901900204B0
:1016D00001C002FF000003FA004003F5008003F0A0
:1016E00000D003EB002004E6007004E100E004DC1D
:1016F000004005D700C005D2004006CD00D006C886
:10170000008007C3003008BE00F008B900C009B46B
:1017100000B00AAF00B00BAA00D00CA500000EA0CC
:1017200000500F9B00C01096005012910000148CC6
:1017300000C0158700B0178200B0197D00D01B785B
:1017400000001E730040206E0090226900F02464A7
:101750000040275F0090295A00E02B5500102E50C2
:101760000020304B0010324600E033410090353C01
:10177000001037370070383200A0392D00B03A28F9
:1017800000A03B2300603C1E00103D1900903D145A
:1017900000103E0F00703E0A00C03E0500003F00F2
:1017A00000403FFBFF803FF6FFC03FF1FF2020508D
:1017B0006C616E6E657242756666657242797465BB
:1017C000733A20002046726565204D656D6F727911
:1017D0003A200020436F6D70696C65643A204F6356
:1017E0007420313320323032330A00204C6173745C
:1017F00020557064617465643A20323032332D3084
:10180000352D3136207C20417574686F723A20285E
:101810006467746168656E6F2C2047656E697573C7
:10182000290A004D61726C696E20322E312E322EE3
:10183000310A0020536F66747761726520526573B8
:1018400065740A00205761746368646F672052658D
:101850007365740A002042726F776E206F75742072
:1018600052657365740A002045787465726E616C08
:101870002052657365740A00506F77657255700A5F
:101880000073746172740A004732385859004D3140
:10189000303031006F6B006572726F722077726941
:1018A00074696E6720746F2066696C650A00446F06
:1018B0006E6520736176696E672066696C652E0AB5
:1018C000004D323900205A3A0020593A0020583A47
:1018D00000656E6473746F7073206869743A2000D9
:1018E00000002200250028002B002E0031003400CB
:1018F00002010000050108010B01050505050705AA
:1019000008080808020202020A0A0808040404047B
:1019100001010101010101010303030303030303A7
:10192000040707070C0C0C0C0C0C0C0C0202020236
:1019300006060606060606060B0B0B0B0B0B0B0B1F
:1019400001021020200808102040102040800201D1
:1019500002010804020101020408102040808040B6
:1019600020100804020180040201804020100804B5
:101970000201080402010102040810204080010253
:1019800004081020408000000A0B02090C0D0E080C
:101990000703040100000000000000000000000038
:1019A0000000000000000000000000000000000037
:1019B00000001211100000000000000000000000F4
:1019C00000000000000000000000000024F404D922
:1019D000201BC40C5C0E9804C4095F0265077101EA
:1019E000F405F900FB04B30048048700C103690053
:1019F0005803550003034500BE023A00840231003B
:101A000053022A002902250004022000E4011C00E0
:101A1000C8011900AF0117009801140084011300D8
:101A2000710110006101100051010E0043010D0011
:101A300036010B002B010B0020010B0015010900E2
:101A40000C01090003010800FB000800F300080076
:101A5000EB000700E4000600DE000600D8000600E8
:101A6000D2000600CC000500C7000500C20005003A
:101A7000BD000400B9000400B5000400B10004007A
:101A8000AD000400A9000400A5000300A2000300AB
:101A90009F0004009B0003009800030095000200D3
:101AA00093000300900003008D0002008B000300F0
:101AB000880002008600020084000300810002000A
:101AC0007F0002007D0002007B000200790002001E
:101AD000770001007600020074000200720001002D
:101AE000710002006F0002006D0001006C00020036
:101AF0006A00010069000200670001006600010041
:101B00006500010064000200620001006100010044
:101B1000600001005F0002005D0001005C00010048
:101B20005B0001005A00010059000100580001004B
:101B3000570001005600010055000100540001004B
:101B40005300000053000100520001005100010049
:101B5000500001004F0001004E0000004E00010047
:101B60004D0001004C0001004B0000004B00010043
:101B70004A0001004900010048000000480001003F
:101B8000470001004600000046000100450000003B
:101B90004500010044000100430000004300010033
:101BA000420000004200010041000000410001002D
:101BB000400001003F0000003F0001003E00000027
:101BC0003E0001003D0000003D0001003C0000001F
:101BD0003C0000003C0001003B0000003B00010015
:101BE0003A0000003A00010039000000390001000D
:101BF0003800000038000000380001003700000005
:101C000037000100360000003600000036000100F9
:101C100035000000350000003500010034000000F0
:101C200034000000340001003300000033000000E5
:101C300033000100320000003200000032000100D9
:101C400031000000310000003100010030000000D0
:101C500030000000300001002F0000002F000000C5
:101C60002F0000002F0001002E0000002E000000B9
:101C70002E0001002D0000002D0000002D000000AE
:101C80002D0001002C0000002C0000002C000000A2
:101C90002C0001002B0000002B0000002B00000096
:101CA0002B0001002A0000002A0000002A0000008A
:101CB0002A0001002900000029000000290000007E
:101CC0002900000029000100280000002800000071
:101CD0002800000028000000280001002700000064
:101CE0002700000027000000270000002700010057
:101CF000260000002600000026000000260000004C
:101D0000260001002500000025000000250000003D
:101D1000250000002500000025000100240000002F
:101D20002400000024000000240000002400010022
:101D30002300000023000000230000002300000017
:101D40002300000023000000230001002200000007
:101D500022000000220000002200000022000000FB
:101D600022000100210000002100000021000000ED
:101D700021000000210000002100000021000100DE
:101D800020000000200000002000000020000000D3
:101D900020000000200000002000000020000100C2
:101DA0001F0000001F0000001F0000001F000000B7
:101DB0001F0000001F0000001F0001001E000000A7
:101DC0001E0000001E0000001E00000024F4D4309D
:101DD00050C38E20C2A24017828B7011127A910DCF
:101DE000816CD90AA861E108C758660761514306AA
:101DF0001E4B5D05C145A7041A411104093D980316
:101E0000713931034036DB0265339102D43054021C
:101E1000802E1D02632CEE01752AC501B028A00199
:101E2000102781018F2564012B244B01E02234010E
:101E3000AC211F018D200D01801FFC00841EED00D0
:101E4000971DDF00B81CD200E61BC600201BBC009B
:101E5000641AB200B219A8000A19A0006A18990001
:101E6000D117910040178B00B516840031167E0003
:101E7000B31579003A157300C7146F0058146A003F
:101E8000EE1366008813630025135E00C7125B0023
:101E90006C12570015125400C111510070114F00FF
:101EA00021114B00D61049008D1047004610440008
:101EB00002104200C00F4000800F3E00420F3C0065
:101EC000060F3B00CB0E3800930E37005C0E35003A
:101ED000270E3400F30D3200C10D3100900D30009B
:101EE000600D2E00320D2D00050D2C00D90C2B009D
:101EF000AE0C2900850C29005C0C2700350C27004E
:101F00000E0C2600E80B2400C40B2400A00B2300B9
:101F10007D0B23005A0B2100390B2100180B2000E8
:101F2000F80A1F00D90A1E00BB0A1E009D0A1D00E8
:101F3000800A1D00630A1C00470A1B002C0A1B00B4
:101F4000110A1A00F7091A00DD091900C40919005D
:101F5000AB091900920917007B09180063091700E3
:101F60004C09160036091600200916000A0915004A
:101F7000F5081500E0081400CC081400B808140097
:101F8000A4081400900813007D0812006B081300C9
:101F900058081200460812003408110023081100E6
:101FA0001208110001081100F0071000E0071000EE
:101FB000D0071000C0071000B0070F00A1071000E5
:101FC00091070E0083070F0074070F0065070E00CE
:101FD00057070E0049070E003B070D002E070E00A5
:101FE00020070D0013070D0006070D00F9060C0071
:101FF000ED060D00E0060C00D4060C00C8060C002F
:10200000BC060C00B0060C00A4060B0099060C00E0
:102010008D060B0082060B0077060B006C060B008A
:1020200061060A0057060B004C060A0042060A0029
:1020300038060A002E060A0024060A001A060A00BC
:102040001006090007060A00FD050900F40509004D
:10205000EB050900E2050900D9050900D0050900D2
:10206000C7050900BE050900B5050800AD05080053
:10207000A50509009C050800940508008C050800CA
:10208000840508007C050800740508006C0507003D
:10209000650508005D050700560508004E050700A8
:1020A000470507004005080038050700310507000F
:1020B0002A050700230507001C0506001605070072
:1020C0000F0507000805060002050700FB040600CF
:1020D000F5040700EE040600E8040600E204070029
:1020E000DB040600D5040600CF040600C904060080
:1020F000C3040600BD040600B7040600B1040500D1
:10210000AC040600A6040600A00405009B0406001B
:1021100095040500900406008A0405008504050066
:10212000800406007A0405007504050070040500AB
:102130006B04050066040500610405005C040500ED
:1021400057040500520405004D040500480405002D
:10215000430405003E0404003A040500350405006C
:10216000300404002C0405002704040023040500A7
:102170001E0404001A0404001604050011040400DF
:102180000D04040009040500040404000004040014
:10219000FC030400F8030400F4030400F00304004B
:1021A000EC030400E8030400E4030400E00304007B
:1021B000DC030400D8030400D4030400D0030400AB
:1021C000CC030400C8030300C5030300281F00005C
:1021D0007A170000BC0F00007B09000047050000D3
:1021E000CC02000071010000BB0000004572726F5C
:1021F000722077726974696E6720746F204545504C
:10220000524F4D210A00DB0FC93F45BCDA3F8FB367
:102210000240FCF0274056946140FE4B9B4084A551
:10222000D840E0231841346A5641E859974164DBAD
:10223000D5416E271742B4B75542CE1A9742C8AE61
:10224000D542B5885A43D40684BFA65FA7BF74435E
:10225000E0BF10B11AC01C2C58C0E8F697C0B849AE
:10226000D6C04E4E17C124D355C1802497C1A0B506
:10227000D5C1121A17C244AE55C2781797C26CACBA
:10228000D5C267885AC320746F6F206C6F6E672049
:10229000657874727573696F6E2070726576656E9D
:1022A0007465640A0020636F6C64206578747275CD
:1022B00073696F6E2070726576656E7465640A006E
:1022C00073686F7700626567696E00507572676545
:1022D0004D6F72650050617573656400436F6E7475
:1022E000696E7565004C6F61642046696C616D654F
:1022F0006E74205400496E736572742066696C6157
:102300006D656E7420616E642073656E64204D315E
:1023100030380A0053656E64204D31303820746FB8
:1023200020726573756D650A00496E73657274205D
:1023300066696C616D656E7420616E642073656E94
:1023400064204D3130380A0052656865617420445C
:102350006F6E6500526568656174696E672E2E2E1A
:102360000052656865617400486561746572205447
:10237000696D656F75740053656E64204D3130383A
:1023800020746F2068656174206E6F7A7A6C650ABC
:10239000004E6F7A7A6C65205061726B65640072D2
:1023A0006573756D6564004469736D69737300527C
:1023B0006573756D696E6700FFFFFF1A151C2418A1
:1023C000241424204500205A0020590020204D3993
:1023D0003220580053746570732070657220756EDA
:1023E000697400220A00556E6B6E6F776E20636F02
:1023F0006D6D616E643A202200486F6D6520257313
:10240000204669727374006F6B0A00526573656EC3
:10241000643A200020453A00205A3A0020593A00F8
:10242000583A00706F7765726F6666005072696E19
:102430007465722068616C7465642E206B696C6CC5
:1024400028292063616C6C6564210A0065AC06B5BF
:1024500011241FBECFEFD1E2DEBFCDBF00E00CBF25
:1024600084B78093F01B14BE0FB6F894A8958091A2
:102470006000886180936000109260000FBE13E0DE
:10248000A0E0B2E0E2EDF6E801E00BBF02C0079089
:102490000D92AE33B107D9F72BE1AEE3B3E001C043
:1024A0001D92A03FB207E1F712E1C7E2D2E100E0DE
:1024B00006C021970109802FFE010E94F4BFC63299
:1024C000D10780E00807A9F70E94A7AD0C9458C374
:1024D0000C940000CF93DF93C6E5D4E120E030E018
:1024E00048E452E4609175177091761780917717E0
:1024F000909178170E9446C287FF13C080E0FE01CA
:10250000C4912091020190E002C095958795CA95EB
:10251000E2F780FD0EC0207120930001DF91CF9182
:102520000895FE01949181E001C0880F9A95EAF721
:10253000E6CF2095F0CF80910608882339F060918E
:10254000D6177091D7178091D817089560E070E082
:1025500080E008954F925F926F927F928F929F9248
:10256000AF92BF92CF92DF92EF92FF920F931F93A1
:10257000CF930091F6071091F7072091F80730915B
:10258000F9078090BD179090BE17A090BF17B0902C
:10259000C0174091FA075091FB076091FC077091BA
:1025A000FD07C090AB17D090AC17E090AD17F0903E
:1025B000AE17C0E1FC01A6EFB7E001900D92CA95FD
:1025C000E1F7E091B717EE2349F1280139014818E6
:1025D00059086A087B08530142010091F6071091DF
:1025E000F7072091F8073091F907080D191D2A1DEA
:1025F0003B1D0093F6071093F7072093F8073093DD
:10260000F907FC0100811181228133810093BD17FC
:102610001093BE172093BF173093C0172091A517B2
:10262000222339F18A019B010C191D092E093F094A
:102630004091FA075091FB076091FC077091FD07EC
:10264000400F511F621F731F4093FA075093FB07FF
:102650006093FC077093FD07FC0184819581A6813E
:10266000B7818093AB179093AC17A093AD17B0933D
:10267000AE17CF911F910F91FF90EF90DF90CF9009
:10268000BF90AF909F908F907F906F905F904F9092
:102690000895EF92FF920F931F93E0924B03F092F5
:1026A0004C0300934D0310934E0360934F037093BC
:1026B0005003809351039FEFFF27621B730B840B22
:1026C00030F4809570956195790B890B99279093DB
:1026D0004A03A6E06A9F00923E03512DEE277A9F9F
:1026E000500DE11D8A9FE00D50933F03E09340039E
:1026F000AFE06A9F00924203512DEE277A9F500D62
:10270000E11D8A9FE00D50934303E0934403AAE048
:102710006A9F00924603512DEE277A9F500DE11DCE
:102720008A9FE00D50934703E09348031F910F9158
:10273000FF90EF90089521E030E0082E02C0220FB4
:10274000331F0A94E2F720953095909106042923CF
:1027500020930604813061F020F0823071F081E036
:1027600008955F9A8091BC088E7F8093BC08F7CF54
:102770008A9A8091BC088D7FF8CF8091080180955E
:10278000817080930601479A8091BC088B7FEDCFC2
:1027900020919C0730919D07F901E95FFB4F9081E3
:1027A00096959695937081E0913009F080E0409184
:1027B00035025091360260919A0770919B074F5FE6
:1027C0005F4F2F5F3F4F2F3291E0390711F430E018
:1027D00020E06217730721F1F901E95FFB4F908157
:1027E00096959695937059F330939D0720939C0787
:1027F00050933602409335024091E5075091E60729
:102800006091DD077091DE07461B570B220F331FC7
:10281000F901EA5CFA4F20813181240F351F0AC08B
:1028200070939D0760939C07509336024093350246
:102830002FEF3FEF3093400220933F020895209105
:10284000980730919907F901E95FFB4F90819370E8
:1028500081E0913009F080E04091370250913802D8
:1028600060919A0770919B074F5F5F4F2F5F3F4FBB
:102870002F3291E0390711F430E020E0621773073E
:1028800011F1F901E95FFB4F9081937069F3309387
:10289000990720939807509338024093370240914C
:1028A000E7075091E8076091DD077091DE07461B4E
:1028B000570B220F331FF901EA5CFA4F2081318157
:1028C000240F351F0AC0709399076093980750939F
:1028D0003802409337022FEF3FEF30933E022093B0
:1028E0003D0208959F92AF92BF92CF92DF92EF92F6
:1028F000FF920F931F93CF93DF9300D01F921F92ED
:10290000CDB7DEB7EFE5F1E10027BB27462F572F04
:10291000A82FAA2341F4A52F542FB85FAA2319F496
:10292000A52F5527B85FA03138F45295A295452FB1
:102930004F70507FA42BBC5FA03428F4550FAA1F02
:10294000550FAA1FBE5FA03818F4550FAA1FB395E4
:10295000550FAA1FEA0FF01F449151E0AA27B85063
:1029600079F1C0F0B0FF02C0440F551FB1FF04C0A1
:10297000440F551F440F551FB2FF06C05295429594
:10298000142F1F70407F512BB3FF1AC0A52F542F57
:10299000442716C0B195B0FF02C055954795B1FFC9
:1029A00004C05595479555954795B2FF05C052957A
:1029B000407F4295452B5F70B3FF02C0452F5527DE
:1029C000DD24CC24BB24B2E0649FD018C108B00A37
:1029D000B00B749FC018B108B00B849FB018B10938
:1029E000659FC018B108B00B759FB018B109859FDD
:1029F000B0196A9FB018B1097A9FB0194D9DA12CEA
:102A000099243327992722275D9DA00C911C301F04
:102A1000901F201FAD9D900C311D901F201F4C9DBD
:102A2000A00C911C301F901F201F5C9D900C311D2D
:102A3000901F201FAC9D300D911D201F4B9D900CB1
:102A4000311D901F201F5B9D300D911D201FAB9DE0
:102A5000900D211D4B9F300D911D201F5B9F900DF0
:102A6000211DAB9F200DB1E0BB24CC24DD24639F4E
:102A7000D018C108B00AB00B739FC018B108B00BD2
:102A8000839FB018B109699FC018B108B00B799F36
:102A9000B018B109899FB019629FB018B109729F2F
:102AA000B019D61AC70AB80A20F0B1E03B0F901F40
:102AB000201F1124792F632F90E0822F0F900F9009
:102AC0000F900F900F90DF91CF911F910F91FF907A
:102AD000EF90DF90CF90BF90AF909F900895AF920E
:102AE000BF92CF92DF92EF92FF920F931F93CF93FB
:102AF000DF93C7E1D4E103ED18E087E2A82E84E17B
:102B0000B82EC12CD12C7601C39469917991899109
:102B100099910E9463B9288939894A895B890E9401
:102B2000C4B90E9468C1F801619371938193919334
:102B30008F01C616D706E806F90610F46B017C0172
:102B4000AC16BD0611F76FEF7FEFCB01A701960121
:102B50000E9489BF2093E3083093E4084093E5087E
:102B60005093E608DF91CF911F910F91FF90EF9066
:102B7000DF90CF90BF90AF900895CF92DF92EF9209
:102B8000FF9280910404882309F457C0C090000488
:102B9000D0900104E0900204F090030420E030E0C3
:102BA000A901C701B6010E945FB9882309F445C095
:102BB00020E030E040E05FE3C701B6010E94C4B905
:102BC0009B01AC010E94C4B92BED3FE049E450E405
:102BD0000E94C4B99B01AC0160E070E080E89FE313
:102BE0000E94FBC06B017C01C092E703D092E80316
:102BF000E092E903F092EA036091170270911802E3
:102C0000072E000C880B990B0E9465B92AE037ED5E
:102C100043E25CE30E94C4B9A70196010E94C4B9D3
:102C200060934F027093500280935102909352022E
:102C3000FF90EF90DF90CF900895C12CD12C80E8C9
:102C4000E82E8FE3F82ED0CF8091C4179091C5174E
:102C5000891B8F7119F490E080E008959091C1175D
:102C6000992351F0833030F48FEF890F19F080935E
:102C7000C117F1CF1092C1178091C51727E5829F28
:102C8000C00111248750974FFC01208120FDE3CF24
:102C90002091C5172F5F2F712093C2173091C51750
:102CA0002091C317321304C02091C2172093C31779
:102CB000089590916F0081E091FD02C080E0089539
:102CC00090916F009D7F90936F000895FC0170813B
:102CD000472F50E0062E02C0559547950A94E2F71B
:102CE00040FF14C04091DA0350E0062E02C0559513
:102CF00047950A94E2F740FF09C021E030E001C0A7
:102D0000220F6A95EAF72095272320830895CF9311
:102D1000DF9324E0829FC0011124EC01C151D94E00
:102D2000FC01E254F74F85529C4FDC012D913D91FF
:102D30004D915C9160817181828193810E941FC05D
:102D4000688379838A839B83DF91CF9108958F92E3
:102D50009F92AF92BF92CF92DF92EF92FF92CF936A
:102D6000DF9320911B02222309F48EC0EC01809195
:102D7000DA03E82E80FF2CC080901D0290901E0286
:102D8000A0901F02B0902002288139814A815B8186
:102D9000C501B4010E9446C2181624F488829982A3
:102DA000AA82BB828090290290902A02A0902B02D6
:102DB000B0902C02288139814A815B81C501B40120
:102DC0000E945FB987FF04C088829982AA82BB8271
:102DD000E1FE2CC08090210290902202A09023025C
:102DE000B09024022C813D814E815F81C501B401E8
:102DF0000E9446C2181624F48C829D82AE82BF8245
:102E000080902D0290902E02A0902F02B090300260
:102E10002C813D814E815F81C501B4010E945FB963
:102E200087FF04C08C829D82AE82BF82E2FE2CC0EE
:102E3000C0902502D0902602E0902702F090280250
:102E4000288539854A855B85C701B6010E9446C23F
:102E5000181624F4C886D986EA86FB86C09031020B
:102E6000D0903202E0903302F09034022885398508
:102E70004A855B85C701B6010E945FB987FF04C020
:102E8000C886D986EA86FB86DF91CF91FF90EF90C6
:102E9000DF90CF90BF90AF909F908F900895CF9389
:102EA000DF93DB01F9019C919130C1F0943080F007
:102EB00094509C938830D1F480819181009771F077
:102EC000019791838083480F591FEA01188206C039
:102ED0008C3539F49C5F9C93943041F4DF91CF9111
:102EE00008958B3339F781E08C93F8CF20813181BD
:102EF000B9016F5F7F4F71836083420F531FEA01F7
:102F00008883808191818F3591056CF7E7CF0F938E
:102F10001F9381E00091E0171091E1172091E217D3
:102F20003091E3174091DC175091DD176091DE1767
:102F30007091DF17041715072607370708F480E09C
:102F40001F910F91089590E080E008952091A603CD
:102F5000833021F425FD0CC024FD0CC030E0A90114
:102F600002C0559547958A95E2F7CA018170089588
:102F700081E0089580E008958091C10384FD0BC035
:102F80008091C30387FD07C09091C403937081E0D3
:102F900019F480E0089581E008952FEB280F2A317D
:102FA00008F047C0E22FF0E08091C1039091C20386
:102FB000A091C303B091C40304C0B695A79597959B
:102FC00087952A95D2F780FD02C081700895E95552
:102FD000FC4FE081EE2341F18091621490916314E3
:102FE000E80FF92FF11D808190ED980F9A3030F0A5
:102FF0008E3251F4818180538A3098F4F093A20389
:10300000E093A10381E008958D3211F08B3249F4F1
:10301000818190ED980F9A3088F38E3211F482817D
:10302000EACFF0E0E0E0EACF1092A2031092A10311
:10303000E9CF80E008958091EB0381110EC02091CB
:10304000190230911A022150310981E0409179171B
:1030500050917A17421753070CF080E008950F93B0
:103060001F938091DD13813019F50E94B693009172
:10307000CE031091CF032091D0033091D103601B78
:10308000710B820B930B28EE33E040E050E00E947E
:1030900089BF6091CA037091CB038091CC0390915A
:1030A000CD03620F731F841F951F1F910F91089509
:1030B0006091D2037091D3038091D4039091D50392
:1030C000D6CF8091DD13813079F482E08093DD13D7
:1030D0000E94B6936093D2037093D3038093D4037A
:1030E0009093D50381E0089580E00895CF93DF9316
:1030F000C0914D17D0914E17209729F16091491733
:1031000070914A1780914B1790914C170E9463C1A0
:103110006E5F7F4F24976C177D07ACF47093130894
:10312000609312080E94B693605A75418F4F9F4F6B
:1031300060931408709315088093160890931708ED
:10314000DF91CF91089510921408109215081092F3
:10315000160810921708F4CF4F925F926F927F92E9
:103160008F929F92AF92BF92CF92DF92EF92FF9297
:103170000F931F93CF93DF93082FEB01C880D98063
:10318000EA80FB8020E030E0A901C701B6010E947F
:103190005FB918160CF079C020E030E040E85FE33A
:1031A000C701B6010E9446C287FF76C029E43AE013
:1031B00046EC52ECC701B6010E94C4B921E931EED8
:1031C00040E852E40E941FC02B013C01A701960178
:1031D000C701B6010E94C4B94B015C012FE237E977
:1031E00042EF50EC0E94C4B9A30192010E941FC09B
:1031F0002B013C01A5019401C701B6010E94C4B98D
:1032000029EF3AE44CE252E40E94C4B9A3019201CE
:103210000E941FC00E9494C16B017C01BFB6F8944C
:10322000C701B6010E9468C1162FA701960160E090
:1032300070E080E093E40E941EC00E9468C101110A
:103240002FC01093BB176093BA1788819981AA8108
:10325000BB818093B3179093B417A093B517B09325
:10326000B617B7FE01C07894DF91CF911F910F91EF
:10327000FF90EF90DF90CF90BF90AF909F908F9096
:103280007F906F905F904F900895C12CD12C80E873
:10329000E82E82E4F82EC2CFC12CD12C7601BECF0D
:1032A0001093A9176093A81788819981AA81BB817F
:1032B0008093A1179093A217A093A317B093A4177C
:1032C000D0CF4091050421E0422768E070E00C94E3
:1032D000DF8F4091050421E042276CE070E00C9400
:1032E000DF8F4091050421E0422764E070E00C94F8
:1032F000DF8F4091050421E0422761E070E00C94EB
:10330000DF8F4091050421E0422761E070E00C94DA
:10331000DF8F4091050421E0422768E070E00C94C3
:10332000DF8F4091050421E042276CE070E00C94AF
:10333000DF8F41E061E070E00C94DF8F41E062E0FC
:1033400070E00C94DF8F4091050421E042270C943B
:10335000DF8F6CE070E00C944F9364E070E00C94AD
:103360004F9362E070E00C944F9361E070E00C9436
:103370004F9361E070E00C944F936CE070E00C941C
:103380004F930F931F93CF93DF930BE214E1C8EE9B
:10339000D8E0F80121913191419151918F0160E084
:1033A00070E080E89FE30E94FBC069937993899362
:1033B0009993F8E0C83FDF0761F70E943C91DF91E5
:1033C000CF911F910F918BCBCF93DF93CDB7DEB70A
:1033D0002C970FB6F894DEBF0FBECDBF19821A82AC
:1033E0001B821C821D821E821F82188619861A86E5
:1033F0001B861C86AE014F5F5F4FBC0183E592E0E8
:103400000E9480922C960FB6F894DEBF0FBECDBFFF
:10341000DF91CF9108958091A1039091A20300972D
:1034200031F04AE050E070E060E00C94BFB760E03B
:1034300070E0CB0108958091A1039091A2030097C1
:1034400031F04AE050E070E060E00C9493B660E048
:1034500070E0CB010895EFDFCB010895ECDF97FD1D
:103460000AC0E9DF6F3F71058105910509F02CF471
:10347000E2DF862F089580E008958FEF0895809110
:10348000A1039091A203892B39F0E8DF91E081112B
:1034900001C090E0892F089591E0FCCFCF93DF9396
:1034A000EC01688170E085E00E943D8E698170E0EA
:1034B00084E00E943D8E6A8170E086E00E943D8E2D
:1034C00088819981482F490F5527551F8A81840F7C
:1034D000952F911D21E0833091050CF420E020937D
:1034E000060803974CF088819981AA818093D617AA
:1034F0009093D717A093D817DF91CF9108958F920B
:103500009F92AF92BF92CF92DF92EF92FF92CF93B2
:10351000DF9300D0CDB7DEB72FEF8417950731F1D9
:103520006A01052E000CEE08FF084C01092E000C64
:10353000AA08BB08681779072CF0CB014617570774
:103540000CF4CA019C01990F440B550B2819390939
:103550004A095B09AFEFB0E00E94C7BFA70196011F
:10356000281939094A095B090E94ABBF80913108CB
:10357000821751F0209331088FEF89831A822095AA
:103580002B83CE0101968ADF0F900F900F90DF9171
:10359000CF91FF90EF90DF90CF90BF90AF909F9032
:1035A0008F9008958F929F92AF92BF92CF92DF92A9
:1035B000EF92FF92CF93DF9300D0CDB7DEB72FEF1E
:1035C0008417950731F16A01052E000CEE08FF08FB
:1035D0004C01092E000CAA08BB08681779072CF0CB
:1035E000CB01461757070CF4CA019C01990F440BF5
:1035F000550B281939094A095B09AFEFB0E00E9461
:10360000C7BFA7019601281939094A095B090E9419
:10361000ABBF80913108821749F02093310829838C
:103620001A828FEF8B83CE01019638DF0F900F90B7
:103630000F90DF91CF91FF90EF90DF90CF90BF90F0
:10364000AF909F908F9008950F930FB70F930091B5
:103650006E000D7F00936E0078940F930BB70F935D
:103660000CB70F921F922F933F934F935F936F93DB
:103670007F938F939F93AF93BF93EF93FF93112407
:1036800088D4FF91EF91BF91AF919F918F917F91DE
:103690006F915F914F913F912F911F900F900CBFB1
:1036A0000F910BBF0F910260F89400936E000F9181
:1036B0000FBF0F911895CF93DF9310923608C1E793
:1036C000D7E1198618860E942FA71A862C98C5E480
:1036D000D7E1198618860ADD1A8680910201807268
:1036E00080930001DF91CF9108958F929F92AF92C6
:1036F000BF92CF92DF92EF92FF920F931F93CF93DF
:10370000DF93B0E4A0E06A2F70E0AB014B0F511DD6
:1037100055954795411119C0EFEAF6E1659174910D
:10372000072E000C880B990B0E9465B9DF91CF9191
:103730001F910F91FF90EF90DF90CF90BF90AF90CF
:103740009F908F900895B42FE0CFA41711F0B41379
:1037500003C0EBEAF7E1E2CF9A0121503109220FD1
:10376000331F220F331FF901E355F94EE590F49012
:10377000F901EF54F94EC591D4918E159F0518F3B8
:10378000A42FC817D90708F4BECFF901E155F94EA7
:1037900005911491F901ED54F94EC590D4908E190C
:1037A0009F09BC0190E080E00E9463B94B015C017D
:1037B000B601601B710B072E000C880B990B0E9441
:1037C00065B99B01AC01C501B4010E94C4B94B01AC
:1037D0005C01CE19DF09BE0190E080E00E9463B970
:1037E0009B01AC01C501B4010E94FBC06B017C01CF
:1037F000B801110F880B990B0E9465B99B01AC01B0
:10380000C701B6010E941FC091CFBC012091E30700
:103810003091E4074091E3075091E40724173507FE
:1038200031F481E02617370709F080E008959A0106
:10383000F1CF0F930FB70F9300916E000F930D7F91
:1038400000936E0000916F000D7F00936F000F9347
:103850000BB70F930CB70F921F922F933F934F9379
:103860005F936F937F938F939F93AF93BF93EF93E8
:10387000FF931124C0D4FF91EF91BF91AF919F911D
:103880008F917F916F915F914F913F912F911F90F9
:103890000F900CBF0F910BBF0F910260F894009333
:1038A0006F000F9100936E000F910FBF0F9118954D
:1038B0008091BD0880FF23C089988FEF8093940783
:1038C0008091BD0881FF1EC08F988FEF8093950770
:1038D0008091BD0882FF19C080910B018095827094
:1038E00080930901439A8FEF809396078091BD08DA
:1038F00083FF13C016988FEF809397070895899AD6
:1039000081E0DCCF8F9A81E0E1CF80910B01827062
:1039100080930901439881E0E7CF169A81E0ECCFCC
:1039200080910604877F80930604129A81E00895AF
:1039300080E00E949B1381E00E949B1382E00E9422
:103940009B13EECF12988091060488608093060442
:103950000895813089F070F0823081F021E030E00C
:1039600001C0220F8A95EAF780910604822B80938A
:10397000060408955F98F2CF8A98F0CF90910801DD
:103980009170909306014798E9CFCF93DF93809190
:10399000EB03811119C0C0911902D0911A0221972D
:1039A00020E030E040E05FE360917517709176179A
:1039B00080917717909178170E941FC00E9463C171
:1039C00021E06C177D070CF020E0822FDF91CF9172
:1039D00008952F923F924F925F926F927F928F92B3
:1039E0009F92AF92BF92CF92DF92EF92FF920F938E
:1039F0001F93CF93DF93CDB7DEB7A0970FB6F894A0
:103A0000DEBF0FBECDBF1C017B015E834D83FC0179
:103A1000EA5BFF4F208131814281538129833A83C0
:103A20004B835C83CA01B9010E9463B94B015C01FD
:103A3000D7012D913D914D915C910E94C4B90E9496
:103A4000E5C02B013C01ED81FE8120813181428165
:103A50005381C501B4010E94C4B90E94E5C06B0145
:103A60007C01C301B2010E9468C169877A878B8794
:103A70009C87683771058105910540F428E730E09F
:103A800040E050E029873A874B875C87C701B60141
:103A90000E9468C16D877E878F87988B6837710514
:103AA0008105910548F428E7C22ED12CE12CF12C98
:103AB000CD86DE86EF86F88AD1019596CD90DD9091
:103AC000ED90FC909897CD82DE82EF82F886F1012E
:103AD000EE5AFF4F6081718182819381611571057A
:103AE0008105910509F49FC10E9465B96D8B7E8B9C
:103AF0008F8B988F9B01AC0160E070E080E89FE3C2
:103B00000E94FBC0698F7A8F8B8F9C8F20E030E002
:103B100040E05FE30E94C4B96B017C01A501940100
:103B2000C501B4010E94C4B92B013C016D857E859D
:103B30008F8598890E9463B99B01AC010E94C4B92A
:103B40009B01AC01C301B2010E941EC0A7019601F6
:103B50000E94C4B94B015C0169857A858B859C857F
:103B60000E9463B99B01AC010E94C4B96D8F7E8F26
:103B70008F8F98A39B01AC01C301B2010E941EC0AC
:103B8000A70196010E94C4B92B013C010E94E5C027
:103B90000E9468C16B017C01C501B4010E9494C1FF
:103BA0000E9468C1698B7A8B8B8B9C8BDC01CB016B
:103BB0008C0D9D1DAE1DBF1D2D813E814F815885F1
:103BC000281B390B4A0B5B0BDA01C901B7FF61C037
:103BD0006D817E818F8198850E9463B9A3019201D6
:103BE0000E941FC0A50194010E941EC020E030E089
:103BF00040E05FE30E94C4B90E94E5C06B017C0114
:103C000020E030E0A9010E9446C218161CF0C12C29
:103C1000D12C7601C701B6010E9468C16B017C01FD
:103C20004D815E816F8178854C155D056E057F0540
:103C300010F46A017B016D817E818F8198856C19FA
:103C40007D098E099F09698B7A8B8B8B9C8BC701B1
:103C5000B6010E9463B94B015C012D893E894F89F1
:103C6000588DCA01B9010E941FC09B01AC01C5015A
:103C7000B4010E94C4B92D8D3E8D4F8D58A10E9474
:103C80001FC00E948CC20E9468C169837A838B83A3
:103C90009C8320E034E244EF59E4698D7A8D8B8D6A
:103CA0009C8D0E94C4B94B015C0169817A818B8132
:103CB0009C8129853A854B855C85621B730B840B3F
:103CC000950B0E9463B9A50194010E94C4B90E949A
:103CD00068C12B013C0169817A818B819C812D8592
:103CE0003E854F855889621B730B840B950B0E9490
:103CF00063B9A50194010E94C4B90E9468C14B0137
:103D00005C013FE6431651046104710408F097C05A
:103D1000F201EE0FFF1FEE0FFF1FED55F04F8591E3
:103D20009591A591B4918C01AD8BBD834FE684161E
:103D30009104A104B10408F08AC0F401EE0FFF1F42
:103D4000EE0FFF1FED55F04F459155916591749120
:103D50009A01CB01D1019996CD92DD92ED92FC9220
:103D60009C9795964D915D916D917C919897C9889E
:103D7000DA88EB88FC884C195D096E097F099D96ED
:103D80004D935D936D937C93D097F101E65BFF4F6C
:103D9000C984DA84EB84FC84C082D182E282F3821B
:103DA000D5964D925D926D927C92D897F10181AE3D
:103DB00092AEA3AEB4AEFD9600831183CD88C282CD
:103DC000DD80D38234962083318382839383C980BC
:103DD000DA80EB80FC80D196CD92DD92ED92FC9260
:103DE000D4973D96CD84DE84EF84F888C082D1825A
:103DF000E282F382A0960FB6F894DEBF0FBECDBF6D
:103E0000DF91CF911F910F91FF90EF90DF90CF90B6
:103E1000BF90AF909F908F907F906F905F904F90EA
:103E20003F902F900895198E1A8E1B8E1C8E198A22
:103E30001A8A1B8A1C8AC12CD12C76012ACFC30175
:103E4000B2010E9472148B018D8B9D836FCFC501CF
:103E5000B4010E9472149B017DCFEFE6F0E08081F7
:103E6000826080830895CF93C82F0E94591694E0F2
:103E7000C99F90011124F901E651F84F2A50384F9B
